:020000040000FA
:1000000085018316F8308500FF23900005308100BC
:10001000951615168312073099008B152030840031
:10002000DF008001840ADF08031D11287620B33029
:1000300081000B110A30BA005F20031D2128B10A8C
:100040001C28102103192628D62021284408310213
:10005000031CD62044083006031930285F202A28C4
:10006000412083203328AB0F0B19232149082B078C
:10007000BC0D48082B07BC0D47082B073C0D85001D
:1000800033285B20B200013E031956283230840029
:10009000840AAE0A0319AF0A5B20800036300406DA
:1000A000031D4828AE0A0319AF0A08002C08AE0049
:1000B0002D08AF0041282F088A002E0882007F20DB
:1000C000013E031968280530AC070318AD0A5F2804
:1000D000B00AAC0A0319AD0A7F20013E0319762845
:1000E0002C08AE002D08AF0003010800B00101305C
:1000F000AD00AF008830AC00AE00FF3808002D081E
:100100008A002C0882003308BB003208B900031DA6
:1001100091283408C7003508C8003608C900AA016C
:1001200008000730AA000130A000A100A200470883
:10013000340203189E28A003A003003CA300480833
:1001400035020318A628A103A103003CA400490816
:1001500036020318AE28A203A203003CA500230820
:1001600024020318BA282308250225080318BF28EB
:100170002308BF28240825022508031C2408003C66
:10018000A900A600A700A800080083169A009B0AF1
:100190001C1555309D00AA309D009C148312080048
:1001A00083169B0A1C141A0883120800C50AC4018E
:1001B000B001C701C801C901E120C508031DDC2841
:1001C0000800450803190800FF3E0319F5288316A7
:1001D0001C0883120239031D08000008C520840A88
:1001E0000408423A0319C50108003008BD00C100E7
:1001F0004708BE00C1074808BF00C1074908C00042
:100200004107003CC1003D30840083169B018312EE
:10021000C50A08000408C6064606C606840008008B
:1002200083169C1811299B01D020C400C300D02044
:10023000C700C307D020C800C307D020C900C30728
:10024000D020430708000108B33E81000B110A21AA
:10025000E1200A21C30803193329B80B3329C30B42
:1002600033290130C500851A3929B70A0319B70A9D
:100270004A29FC30370703183F29B7014A295F2074
:100280004120C701C801C90183200A30BA00B70163
:100290000830C300AA0803197C29B90B08003208EA
:1002A000B90034084706031D57292A105F2923087F
:1002B000A607031C5F292908A6072008C7073508D9
:1002C0004806031D6529AA106D292408A707031CE9
:1002D0006D292908A7072108C80736084906031D04
:1002E00073292A1108002508A807031C08002908FB
:1002F000A8072208C9070800BB0803198529BA0BFB
:1003000008000A30BA00BB0B080041208320080017
:1003100000340034053400345034033400343C34A9
:100320000034503400340134FF340034503400348D
:1003300000343C3400345034033400340534003489
:100340005034003401340534FF3450340034023466
:10035000053400345034003401340534FF34503453
:10036000FF34003400340534003450340334003496
:100370003C340034503400340134FF340034503401
:10038000003400343C340034503403340034053439
:1003900000345034003402340534FF345034FF3418
:1003A00000340034053400345034043400343C3418
:1003B0000034503400340234FF34003450340034FC
:1003C00000343C34003450340434003405340034F8
:1003D0005034003401340534FF34503400340334D5
:1003E000053400345034003401340534FF345034C3
:1003F000FF34003400340534003450340434003405
:100400003C340034503400340134FF340034503470
:10041000003400343C3400345034043400340534A7
:1004200000345034003402340534FF345034FF3487
:10043000003400340534003450340434003428349B
:100440000034503400340234FF340034503400346B
:10045000003428340034503404340034053400347B
:100460005034003401340534FF3450340034023445
:10047000053400345034003401340534FF34503432
:10048000FF34003400340534003450340634003472
:1004900032340034503400340234FF3400345034E9
:1004A000003400343234003450340734003405341E
:1004B00000345034003401340534FF3450340034F7
:1004C0000234053400345034003401340534FF3430
:1004D0005034FF3400340A341E34053450340034B0
:1004E0000834FF3405345034003401341E34FF34F2
:1004F000503400340F341E34053450340034083482
:10050000FF3405345034003401341E34FF34503489
:10051000003402341E3405345034003401341E34A7
:10052000FF345034FF3401340134053405340534CC
:0E05300001340134803480348034FF34FF34D1
:02400E00A43FCD
:10422000520043006E00610076006C006900670078
:104230006800740073002E00610073006D002000A0
:10424000300032002F00300036002F0032003000E6
:10425000310032002000520031002E0030002E00CC
:104260003000280063002900200050006500740021
:104270006500200047007200690066006600690062
:1042800074006800730020003200300030003600F7
:104290002D003200300031003200200069006E0035
:1042A00066006F00400070006900630070007200DB
:1042B0006F006A0065006300740073002E006F00D9
:0A42C000720067002E0075006B000D
:00000001FF
